:020000020000FC
:020000000EC030
:020006004AC0EE
:10001C0024C00FEF01BB0FEF02BB00E004BB00E3F9
:10002C0005BB0FEF07BB0FEF08BB0FE50DBF04E0DF
:10003C000EBF51E00EE005BD0CE003BD00E809BFAA
:10004C0000EC07B90BE806B900E905BF789400E8A5
:10005C0008B9FFCF78948895089504B115B120E0C4
:10006C0030E040E0043618F4113008F404C00456B3
:10007C0010404395F7CF4A3038F40A3018F00A5044
:10008C003395FBCF202F03C02FEF3FEF4FEF189589
:10009C0008D05A9529F453E06A9511F469E1DADF36
:1000AC00189500E008BB513021F0523041F053302C
:1000BC0079F0022F16D002BB01E008BB0895032F84
:1000CC0010D013B314FF005802BB02E008BB089514
:1000DC00042F07D013B315FF005802BB04E008BB74
:1000EC0008950030A1F00130A1F00230A1F00330EE
:1000FC00A1F00430A1F00530A1F00630A1F00730DA
:10010C00A1F00830A1F00930A1F00FEB089500EC3C
:10011C00089509EF089504EA089500EB089509E99C
:10012C00089502E9089502E8089508EF089500E89B
:06013C00089500E908959A
:00000001FF
